S01800006275696C642F6D696361322F6D61696E2E737265632D
S11300000C94B5010C94D2010C94D2010C94D2013D
S11300100C94D2010C94D2010C94D2010C94D20110
S11300200C94D2010C94D2010C94D2010C94D20100
S11300300C94D2010C94D2010C94D2010C947E1C29
S11300400C94D2010C943B020C9464020C94D201E3
S11300500C948E020C9452190C94D2010C94D2017B
S11300600C94D2010C94D2010C94C5230C94D201AB
S11300700C94D2010C94D2010C94D2010C94D201B0
S11300800C94D2010C94D2010C94D20100060030DD
S1130090003C0090010F01F803D9079B0F060000F4
S11300A0000A00190032006400C8019003200640D1
S11300B03158000057F685035544020F60E0261CB2
S11300C06B55700100000000000000000081013148
S11300D07C00007BF9AE02388C3280401026A16B84
S11300E0551001000000000000000000F301315130
S11300F0000050F74F030E44020F58E026A16B5541
S113010070010000000000000000008101315CE08B
S1130110005CDB4201AA8C3280301026A16B5510A2
S113012001000000000000000000F3013145600000
S11301304555BB039C80020F68E026A16B547001F7
S11301400000000000000000008101315800005749
S1130150F685035590020F60E026A16B55700100EF
S11301600000000000000000810100002110422076
S113017063308440A550C660E770088129914AA184
S11301806BB18CC1ADD1CEE1EFF1311210027332FB
S11301905222B5529442F772D662399318837BB3D4
S11301A05AA3BDD39CC3FFF3DEE36224433420048B
S11301B00114E664C774A44485546AA54BB5288524
S11301C00995EEE5CFF5ACC58DD5533672261116DB
S11301D03006D776F6669556B4465BB77AA7199774
S11301E03887DFF7FEE79DD7BCC7C448E558866863
S11301F0A7784008611802282338CCC9EDD98EE9C4
S1130200AFF9488969990AA92BB9F55AD44AB77A3A
S1130210966A711A500A333A122AFDDBDCCBBFFB13
S11302209EEB799B588B3BBB1AABA66C877CE44C4A
S1130230C55C222C033C600C411CAEED8FFDECCD63
S1130240CDDD2AAD0BBD688D499D977EB66ED55E1A
S1130250F44E133E322E511E700E9FFFBEEFDDDFB3
S1130260FCCF1BBF3AAF599F788F8891A981CAB13F
S1130270EBA10CD12DC14EF16FE18010A100C23071
S1130280E3200450254046706760B9839893FBA32C
S1130290DAB33DC31CD37FE35EF3B1029012F322C1
S11302A0D2323542145277625672EAB5CBA5A8957C
S11302B089856EF54FE52CD50DC5E234C324A01411
S11302C081046674476424540544DBA7FAB799870C
S11302D0B8975FE77EF71DC73CD7D326F236910661
S11302E0B01657667676154634564CD96DC90EF954
S11302F02FE9C899E9898AB9ABA9445865480678B1
S11303002768C018E1088238A3287DCB5CDB3FEB6B
S11303101EFBF98BD89BBBAB9ABB754A545A376A00
S1130320167AF10AD01AB32A923A2EFD0FED6CDD3B
S11303304DCDAABD8BADE89DC98D267C076C645C50
S1130340454CA23C832CE01CC10C1FEF3EFF5DCF4B
S11303507CDF9BAFBABFD98FF89F176E367E554EA0
S1130360745E932EB23ED10EF01E11241FBECFEF49
S1130370D0E1DEBFCDBF14E0A0E0B1E0E0E1F0E603
S113038000E00BBF02C007900D92A433B107D9F768
S113039018E0A4E3B4E001C01D92A639B107E1F767
S11303A00C94D2020C940000AF92BF92CF92DF92D1
S11303B0EF92FF920F931F93CF93DF9306EEA090DB
S11303C05408B0905508C0905608D0905708A1140E
S11303D0B104C104D104C9F110E068EC75E0EE2465
S11303E0FF2481E090E0A0E0B0E00E2C04C0880F70
S11303F0991FAA1FBB1F0A94D2F78A219B21AC2103
S1130400BD210097A105B10579F0202F332744279A
S11304105527FB0185819681A781B08582179307B3
S1130420A407B5070CF405811F5F0894E11CF11CB7
S1130430675F7F4F1830A8F28FB7F894992712B7E7
S11304401D5F011728F4012F03C08FB7F894992773
S11304500093C20601BF109253068FBF0E946A0820
S1130460DF91CF911F910F91FF90EF90DF90CF908C
S1130470BF90AF9008951F920F920FB60F92112460
S11304802F933F934F935F936F937F938F939F9398
S1130490AF93BF93EF93FF939FB1809149058FB9B9
S11304A0892F0E947C1DFF91EF91BF91AF919F9185
S11304B08F917F916F915F914F913F912F910F9009
S11304C00FBE0F901F9018951F920F920FB60F92A8
S11304D011242F933F934F935F936F937F938F9345
S11304E09F93AF93BF93EF93FF935F9B06C08CB131
S11304F040E050E060E00E941125FF91EF91BF9130
S1130500AF919F918F917F916F915F914F913F91A7
S11305102F910F900FBE0F901F90189578941F92F3
S11305200F920FB60F9211242F933F934F935F9323
S11305306F937F938F939F93AF93BF93EF93FF93A7
S11305400E94DD26FF91EF91BF91AF919F918F9112
S11305507F916F915F914F913F912F910F900FBEBB
S11305600F901F901895BC018FB7F894482F55270A
S113057020914E06E22FFF27EE0FFF1FEE5FFA4F8A
S113058080819181892B51F42F5F277020934E062F
S1130590608371834FBF81E090E008954FBF80E096
S11305A090E00895CFEFD0E1DEBFCDBFD698A79AF3
S11305B0A69AA59AA49AA39AA29AA19AA09A8C9A66
S11305C08F9A8E9ABB98BF98D498DC9883E08C5FFE
S11305D08739E8F390E08AE08093DB0490934E0639
S11305E090936C0582E095E0FC019C01225F3F4FF3
S11305F011921192029628173907D4F70E94D10656
S11306000E94D1060E94D1060E9400078FB7F89479
S1130610992710925F068FBF8FB7F894682F7727BA
S113062082E08093D004809337048CE895E0909323
S11306305206809351061092900582E290E09093C6
S11306403F0680933E061092FB0410923D061092E2
S11306505D0810925C081092F4041092F304109256
S1130660140510921305109260081092B3041092AE
S11306709E041092D80610923C0681E090E080938C
S113068016058CE291E09093B5068093B4062FEFA3
S11306903FEF3093B1062093B0063093B306209316
S11306A0B206109215051092A4041092BF0610927F
S11306B0DA0480E291E09093B8058093B705109234
S11306C09F041092D7061092D606109270051092CD
S11306D06F05109245061092440680E090E0A0E079
S11306E0B0E08093CC049093CD04A093CE04B09357
S11306F0CF041092C1051092C2051092C305109246
S1130700C40580E290E09093F2048093F104909306
S1130710DF048093DE0482E390E0909335088093B5
S1130720340880E496E09093C0058093BF059093CD
S11307302F0880932E0810921408109236081092F5
S1130740B90510924D06109219051092E104109209
S1130750E004109225081092240810923904109293
S1130760380410924106109240064EED4093130651
S1130770309312062093110685E0809315069DE7B9
S11307809093140610923406109233064093E706B1
S11307903093E6062093E5068093E9069093E806F5
S11307A010920807109207078FED80931E0530936F
S11307B01D0520931C0587E08093200590931F0559
S11307C010923F0510923E051092160680915B062A
S11307D090915C069093180680931706809100010F
S11307E09091010190931A06809319066FBF28E037
S11307F0E4EBF4E080E291E081939193215027FFB0
S1130800F9CF8FB7F8949927B998BB98BA986B9891
S11308106A986F9A6E9A8FBF81E480938A00D69803
S11308208C9A8E9A8F9A949A979A969A6AE380E011
S11308300E9444076BE380E00E94440780ED97E048
S113084000000000000000000000000000000000A4
S1130850019718161906A4F380E880935505682FAC
S11308608BE00E94440780E980935705682F84E059
S11308700E944407109259058FE680935A0585E536
S113088080935B05609159058FE00E944407809135
S11308905A05682F80E10E94440780915B05682F08
S11308A081E10E94440711E010935D05612F83E10B
S11308B00E944407109368058AE495E0DC011196D0
S11308C0E1EBF0E09C01225E3F4F84918D933196E1
S11308D02A173B07D4F711E0CBE4D5E08991682FC0
S11308E0812F0E9444071F5F1D30C0F380915C0577
S11308F0682F82E10E94440760E08BE00E94440775
S11309006FE382E40E94440761E180E00E944407AF
S113091066EA8EE00E9444078EE00E94680783FF27
S1130920FBCF66E28EE00E94440761EE80E00E9405
S1130930440780916705682F89E00E94440760E0BE
S11309408BE00E94440766EA8EE00E944407CEE0F2
S11309508C2F0E94680783FFFACF66E28C2F0E94D7
S1130960440780E980935705682F8DE00E9444076F
S113097080916805809327080E949B078FB7F8949D
S11309809927109215088FBF8FB7F894282F332713
S113099010927405109273051092500610924F062F
S11309A010929208109291081092C7051092C605F1
S11309B08DE791E0A0E0B0E0809358089093590847
S11309C0A0935A08B0935B082FBF0E949B078FB770
S11309D0F8949927C6B917B88FBF8FB7F894482FE2
S11309E05527209100013091010181E597E3289F6B
S11309F0B001299F700D389F700D1124CB018F5ABF
S1130A00984C9093D3068093D20690936208809377
S1130A10610885E89FE0289FB001299F700D389FE9
S1130A20700D1124CB018B57904F9093DD0480936C
S1130A30DC044FBF0E94D106809100019091010116
S1130A4090933D0880933C081092530810922D080F
S1130A5010922C081092BD051092BC058FB7F89423
S1130A60182F80E0C5E7D5E0AEE3B8E0E0E6F6E0B5
S1130A709FEF90839183928313829D9399938F5FC9
S1130A8034968431A8F39093A60480910001809356
S1130A90A5049093A7049093A80410928B05109238
S1130AA06B0510924A069093C50510923604109275
S1130AB0CA041092340410925E0884E690E0909385
S1130AC09804809397048CED95E09093D8048093D8
S1130AD0D70488EE93E09093390880933808909374
S1130AE0BB058093BA051092F50481E08093290830
S1130AF08093D5061092D9048093130780E398E07D
S1130B000E94B6072091300830913108809100018D
S1130B1090910101280F391F81E597E3289FA001D7
S1130B20299F500D389F500D1124CA018F5A984C9B
S1130B30909322088093210885E89FE0289FB001C4
S1130B40299F700D389F700D1124CB018B57904F46
S1130B509093900880938F08109210061092930837
S1130B60109246061092BE061092FA041092E20405
S1130B701092C3061092B606109210071092350414
S1130B80109290008FE089B982E08BB986E080935F
S1130B9095008CB188E08AB91FBF0E9400071092AB
S1130BA090008FE089B982E08BB986E0809395004C
S1130BB088ED8AB98FB7F89499274091D0048FBFF4
S1130BC06FEF7FEFA3E08FB7F894282F332780913E
S1130BD07D008F7E80937D008BE080938A0010924D
S1130BE089001092880070938700609386001092A9
S1130BF08B0080918B00806480938B00139A1092F9
S1130C008C0080917D00806180937D002FBF1092C5
S1130C10E304423009F07DC08FB7F894482F55277C
S1130C20E0915106F09152061482A093D0041092E0
S1130C309E041092B3047093B1066093B0061092B0
S1130C40BE051092BF06EEE9F0E084919927382F93
S1130C502227319684919927282B392B30935E06CD
S1130C6020935D06ECE8F0E084919927382F222741
S1130C70319684919927282B392B3093EA042093B9
S1130C80E9044FBFE0915106F091520614828FB7E8
S1130C90F8949927A093D0048FBF6BE380E00E945F
S1130CA0440769E380E00E94440788EC90E0000078
S1130CB00000000000000000000000000000019798
S1130CC018161906A4F3BB98BA980E94DB07809102
S1130CD03D068F3128F020E03AE040E050E004C0C7
S1130CE020E830E040E050E060E084E00E94FA0751
S1130CF080EC8DB9B8980E946A088091BF06882359
S1130D0041F020E03AE040E050E061E085E00E94FC
S1130D10FA0728EE33E040E050E060E083E00E9410
S1130D20FA07109253080E946A0810928B050E94D9
S1130D307C0864EF71E00E94D22FAA27BB279C0194
S1130D40AD0161E0862F0E94FA0720E335E740E019
S1130D5050E061E080E00E94FA078FEF8093550530
S1130D6078948FB7F894482F552790916C05E92F04
S1130D70FF27EE0FFF1FEE5FFA4F2081318121150F
S1130D80310529F47894889500000000EACF108298
S1130D9011829F5F977090936C054FBFF90109957D
S1130DA0E0CF1092540810925508109256081092F1
S1130DB05708109253068FEF80935F088093940432
S1130DC01092FC0483E08093560696EE9093C2063C
S1130DD08FB7F894282F332787B78E7F87BF87B7BD
S1130DE08D7F87BF80B7886080BF8BE083BF12BED2
S1130DF091BF87B7826087BF2FBF81E090E00895DD
S1130E008FB7F894682F80E090E04CE354E09C01A5
S1130E10F901E80FF91FEC53F94F4483558312820B
S1130E201382118201962B5F3F4F455D5F4F8230E5
S1130E30910574F31092260810924306109242060C
S1130E401092D6041092D50410923B0410923A04E6
S1130E501092930410929204109223081092B706F1
S1130E60109228081092E6041092E50410921805D6
S1130E70109217058091C8069091C9069093DF06D9
S1130E808093DE066FBF0895880F949896E087FFDD
S1130E9002C0979A01C097989698969A880F915095
S1130EA097FFF5CF979A9698969A949A97E067FF4A
S1130EB002C0979A01C097989698969A660F915097
S1130EC097FFF5CF949A979A969A81E090E00895C7
S1130ED090E0880F949826E030E087FF02C0979A4C
S1130EE001C097989698969A880F2150304037FF02
S1130EF0F4CF27E030E097989698969A8F98949A32
S1130F00969840E050E0879941E0892F9927215035
S1130F103040442329F0880F991F982F916002C014
S1130F20982F990F969A37FFEBCF949A8F9A979AA6
S1130F30892F992708958FB7F894282F8091E40476
S1130F40882391F480E090E0E5E1F8E08193019654
S1130F508C309105DCF38EE180931F088FE1809340
S1130F60200881E08093E4042FBF0895FC018FB72B
S1130F70F894282F332780918800909189008083EA
S1130F80918380917C0084FF0EC08091B104909184
S1130F90B20401969093B2048093B10480917C00D2
S1130FA0806180937C008091B1049091B20482832B
S1130FB093832FBF089580915305682F89E00E9481
S1130FC0440760E08BE00E94440761E180E00E94F6
S1130FD044078DE790E000000000000000000000DE
S1130FE0000000000000019718161906A4F381E020
S1130FF090E00895EF92FF920F931F93CF93DF93A6
S1131000962F79018A01883050F4623044F46623C3
S113101049F423E0E216F1040105110518F480E017
S113102090E051C0682F7727FB0153E0EE0FFF1FBC
S11310305A95E1F7E60FF71FE853FA4FE182F2827F
S11310400383148390838FB7F894C82FDD2782B766
S1131050E80EF11C011D111DE582F682078310873D
S113106021E030E040E050E004C0220F331F441F71
S1131070551F6A95D2F78091540890915508A09114
S11310805608B0915708822B932BA42BB52B809331
S1131090540890935508A0935608B093570880912C
S11310A0C2069927AA27BB27E816F9060A071B07D1
S11310B038F4E092C206E1BE109253060E946A0818
S11310C0CFBF81E090E0DF91CF911F910F91FF900E
S11310D0EF9008958091080118162CF089E499E2A4
S11310E00E94B30206C085B7837E85BF85B7806240
S11310F085BF80E090E008958FB7F894482F552776
S11311002091210830912208832F881F8827881F67
S1131110220F331F882321F08BE090E12827392701
S11311202F5F3F4F309322082093210880918F082E
S113113090919008282739274FBFC90108954F92ED
S11311405F926F927F928F929F92AF92BF92CF9253
S1131150DF92EF92FF920F931F93CF93DF93CDB75C
S1131160DEB7A8970FB6F894DEBF0FBECDBF3C0123
S113117020910001309101018091BC059091BD0541
S113118001969093BD058093BC05F30182A193A1C0
S1131190019709F0CDC4938180910201981709F059
S11311A0C7C480819181FFEF8F3F9F0721F0821791
S11311B0930709F0BDC4F301928183E08C5F8B3205
S11311C0E8F3892F99278232910509F46AC383329F
S11311D091055CF48032910509F42BC181329105AB
S11311E00CF010C24F9789F09FC48432910509F422
S11311F09BC3843291050CF458C38532910509F4DC
S1131200C2C3869709F412C48FC490918B059923A5
S113121009F08AC48FB7F894982E15E0A12EB12C4A
S1131220A60CB71CF3010581D0900001192FC92E1B
S113123020E030E0AE014F5F5F4FFA01E20FF31F91
S1131240BE016B5E7F4FDB01A20FB31F8FEF8C9348
S113125080831F5F2F5F3F4F143160F310E0F5016F
S11312608181181770F4E12FFF27DA01AE0FBF1F39
S1131270EA0DFB1D82818C931F5FF5018181181794
S113128090F390E0143170F49B01290F311DD501C6
S1131290A10FB11D12968C91F90180831F5F9F5F8E
S11312A0143190F344E1BE016F5F7F4F8D2D0E9496
S11312B0B00D8F5F9F4F21F144E165E775E0802F0A
S11312C00E94B00D8F5F9F4F59F06EE378E0802F3E
S11312D00E94C40D65E775E0802F0E94FD0E7BC05F
S11312E044E16EE378E0802F0E94B00D8F5F9F4F42
S11312F009F068C06EE378E0802F0E94C40D62C0DC
S1131300B5E1EB2EF12CEC0EFD1E44E1B7018D2D61
S11313100E94B00D8F5F9F4F59F144E165E775E07E
S1131320802F0E94B00D8F5F9F4F59F06EE378E0DD
S1131330802F0E94C40D65E775E0802F0E94FD0E8A
S113134041C044E16EE378E0802F0E94B00D8F5FCE
S11313509F4F09F040C044E16EE378E0802F0E9483
S1131360B00D8F5F9F4FB9F544E165E775E030C07C
S113137044E1BE016F5F7F4F8D2D0E94B00D8F5FE2
S11313809F4F49F544E1B7018D2D0E94B00D8F5F49
S11313909F4F09F544E165E775E0802F0E94B00D89
S11313A08F5F9F4F31F465E775E0802F0E94C40D75
S11313B012C044E165E775E0802F0E94B00D8F5F95
S11313C09F4F19F0A1E0CA2E06C044E16EE378E015
S11313D0802F0E94B00DCC2031F080918B058823A2
S11313E011F00E942A0F10E0CC24DD24F5E1EF2E49
S11313F0F12CEC0EFD1EEC0CFD1C44E16EE378E0D8
S1131400F70180810E94B00D8F5F9F4F29F462E045
S1131410F70180810E94E9121F5F0894C11CD11C4E
S1131420143120F362E0F50180810E9440139FBED5
S11314307BC383010B5F1F4FF3018581C82EDD241D
S113144061E08C2D0E9485138F5F9F4F09F46CC35C
S11314508FB7F894A82EF80187819085A185B2856D
S11314608093FE049093FF04A0930005B0930105BC
S1131470BB24F30180898F3FD1F07801EB0CF11C80
S113148061E0F70183850E9485138F5F9F4F29F4E4
S113149062E0F70183850E94E912B394F3E1FB153E
S11314A030F0F801EB0DF11D83858F3F31F720916A
S11314B0C505822F9927C816D90649F130918B05A5
S11314C0832F8150823018F58FB7F894182F8091AC
S11314D0F5048823D1F48091000180936808309347
S11314E069088091B60680936B0820936A088C2D56
S11314F0992723E638E044E0BC0183E20E94BA0F56
S11315009927813011F48093F5041FBF79C090911D
S11315108B05933021F080914A06882321F1809134
S11315204A06882319F482E00E94A11282E0809383
S11315308B0510923404C092C505F8018481992763
S113154025813681829FA001839F500D929F500D6B
S11315501124CA01820F931F880F991F9093BB0512
S11315608093BA0530C0923009F04AC0822F99277F
S1131570C816D90609F044C0F80184819927258149
S11315803681829FA001839F500D929F500D11249C
S1131590CA01820F931F880F991F9093BB058093F4
S11315A0BA05055F1F4F44E1B801809100010E9414
S11315B0B00D8F5F9F4F19F400E010E002C001E00E
S11315C010E0002379F00E947C0864E670E00E9439
S11315D0D22FAA27BB279C01AD0161E0862F0E9470
S11315E0FA070EC08091BA059091BB05AA27BB27C4
S11315F09C01AD0161E0862F0E94FA070093340438
S1131600AFBE92C25524E5E0AE2EB12CA60CB71C99
S113161061E0F30185810E9485136C018F5F9F4F08
S113162009F482C28FB7F894482EF52C850161E045
S1131630F80184810E9485138F5F9F4F29F462E033
S1131640F80184810E94E9126F2DF80184810E94BF
S11316505014F3940F5F1F4FF3E1FF1540F780918F
S11316604A06882329F08091A6040E94B01317C16A
S113167090918B05892F8250823038F48FEF0E942D
S1131680B01381E08093D9040AC1913009F007C1F5
S1131690F601EE0FFF1FEE0FFF1FE05AF94F838193
S11316A082FD03C08460838301C0592E8091130797
S11316B0882309F4D5C080E398E00E94B60780919E
S11316C0300890913108A0913208B0913308F501A7
S11316D0208D318D428D538DBC01CD010E947E142D
S11316E06B017C01C701AA2797FDA095BA2FBC0105
S11316F0CD010E94092FF7FE06C020E030E040E84B
S113170057E40E945C2E22E538E34EE054E40E9444
S1131710782F4B015C01C601AA2797FDA095BA2F2B
S1131720BC01CD010E94092FD7FE06C020E030E0A5
S113173040E857E40E945C2E2FE836E34EE05CE379
S11317400E94782FDC01CB019C01AD01C501B401DD
S11317500E945C2EDC01CB0120E030E040E05FE33E
S1131760BC01CD010E94782FDC01CB0120E030E0E8
S113177040E05FE3BC01CD010E94782F6B017C0146
S11317800091970410919804C801AA2797FDA09589
S1131790BA2FBC01CD010E94092F17FF06C020E01B
S11317A030E040E857E40E945C2E20E030E040E066
S11317B05FE30E94782FDC01CB019C01AD01C701DE
S11317C0B6010E945C2EDC01CB01BC01CD010E945C
S11317D0EC2EDC01CB01909398048093970490E065
S11317E0292F809160068F3FC9F0E22FFF27EE0F6B
S11317F0FF1FEE0FFF1FE05AF94F838180FD9F5FAB
S11318002F5F243158F4E22FFF27EE0FFF1FEE0F56
S1131810FF1FE05AF94F80818F3F39F7892F9927AD
S11318202091970430919804289FA001299F500D7E
S1131830389F500D1124CA01820F931F820F931FEA
S1131840880F991F9093D8048093D704220F331FD5
S1131850220F331F3093390820933808109213074E
S11318600E949214882359F480914A06882339F4FB
S11318700E94B8140E9439150E942C1610C05520DD
S113188071F48091380890913908AA27BB279C01EC
S1131890AD0161E0862F0E94FA0750925E084FBEA8
S11318A043C1C3010E94DB1340C110918B05113069
S11318B009F03AC18FB7F894082F812F0E94A11222
S11318C08FEF0E94B0131093D90490E080916006CA
S11318D08F3FD9F0E92FFF27EE0FFF1FEE0FFF1FF9
S11318E0E05AF94F838180FF02C08B7F83839F5F1F
S11318F0943158F4E92FFF27EE0FFF1FEE0FFF1F5F
S1131900E05AF94F80818F3F29F783E080938B055C
S11319101092350428EE33E040E050E061E082E0CC
S11319200E94FA070FBF00C183010B5F1F4F61E0E4
S1131930F30185810E9485138F5F9F4F09F4F4C0E2
S1131940F8014581242F33278091000190910101F2
S11319502817390709F4E8C08FB7F894F82E809156
S11319608B05823049F48091C505481729F4F301A9
S11319704583C3010E94DB13F801648185810E94C1
S11319805014FFBED1C080914A06882309F4CCC00C
S11319908FB7F894E82E05E0C02ED12CC60CD71CC6
S11319A061E0F30185810E948513DC018F5F9F4F05
S11319B051F0AA0FBB1FAA0FBB1FA05AB94FF601C3
S11319C0818111968C93FF248301085F1F4F63E08C
S11319D0F80181918F010E948513FC018F5F9F4F55
S11319E039F0EE0FFF1FEE0FFF1FE05AF94FF1829F
S11319F0F39443E14F1558F780918B05843069F4D3
S1131A0085E080938B050E94311720E335E740E0A1
S1131A1050E061E080E00E94FA07F60182818823A9
S1131A2019F481E00E94FF17EFBE7EC080918B0500
S1131A30863029F080916B05882309F475C08FB72F
S1131A40F894C82EF5E0EF2EF12CE60CF71C61E0BB
S1131A50F30185810E948513A82FBB27AA0FBB1F02
S1131A60AA0FBB1FA05AB94FF701818112968C931C
S1131A70DD24F30180858F3F09F445C087010D0DF6
S1131A80111D63E0F80183810E948513FFEF8F3FEE
S1131A909F0771F1DC01AA0FBB1FAA0FBB1FA05A3D
S1131AA0B94FF801828912968C9312971FB7107858
S1131AB0F89499279F938F938C9199279F938F9351
S1131AC089E091E09F938F9384E197E09F938F93B4
S1131AD00E94080E4DB75EB7485F5F4F0FB6F8948B
S1131AE05EBF0FBE4DBF0E94DC0E112309F0789437
S1131AF0D3945EE05D1538F0F701ED0DF11D83819F
S1131B008F3F09F0BBCF80918B05853029F486E0A7
S1131B1080938B050E947018F7018281823019F43A
S1131B2083E00E94E318CFBEC301009709F03C0193
S1131B30C301A8960FB6F894DEBF0FBECDBFDF91E8
S1131B40CF911F910F91FF90EF90DF90CF90BF90B6
S1131B50AF909F908F907F906F905F904F9008957B
S1131B60582F90E0941768F4292F3327FB01E20FD4
S1131B70F31F8081851711F4C90108959F5F94179D
S1131B8098F38FEF9FEF08951F93CF93482FDB01B6
S1131B90282F3327809100019091010128173907DC
S1131BA0A1F18FB7F894C82F80E09C919F3F69F012
S1131BB0941759F08F5F843140F4FD01E80FF11D53
S1131BC0E081EF3F11F0E417A9F78431B9F41FB7AE
S1131BD01078F8948DE291E09F938F9384E197E0DD
S1131BE09F938F930E94080E0E94DC0E0F900F901B
S1131BF00F900F90112341F0789406C0FD01E80F77
S1131C00F11D808184134083CFBFCF911F9108952C
S1131C108F929F92AF92BF92CF92DF92EF92FF92F8
S1131C200F931F93CF93DF93CDB7DEB7C054D0404B
S1131C300FB6F894DEBF0FBECDBF6196EEACFFAC1D
S1131C4061976396CEACDFAC639723E5A22EB12CEB
S1131C50AC0EBD1ED601ED916D01E53261F0EE23AF
S1131C6009F494C0D701ED937D011C92D601ED9146
S1131C706D01E532A1F720E0D601ED916D018E2FC3
S1131C8099278F369105B1F18037910574F4833625
S1131C909105C9F08436910524F483359105F1F05A
S1131CA018C08936910579F114C08537910561F121
S1131CB08637910524F48337910581F00AC088376B
S1131CC0910531F106C0F50182E090E0A80EB91E3D
S1131CD0E081D701ED937D011C92BCCFF50182E038
S1131CE090E0A80EB91E00811181B801C7010E94BD
S1131CF0502EB0CF98E0892E912C80E3D7018D939C
S1131D007D012C9308C021E08AE0882E912C03C029
S1131D1000E1802E912CF50182E090E0A80EB91E1E
S1131D200190F081E02D222351F0F7FF08C0F095D7
S1131D30E195FF4F8DE2D7018D937D011C928E01B9
S1131D400F5B1F4FD8011E928D01CF01B4010E9479
S1131D50D22F282F205D2A330CF0295DD8012E9331
S1131D608D01CF01B4010E94D22FFB01672B69F7CB
S1131D70B801C7010E94502EF80101900020E9F734
S1131D803197E01BF10BEE0EFF1E64CF80E090E074
S1131D90C05CDF4F0FB6F894DEBF0FBECDBFDF913E
S1131DA0CF911F910F91FF90EF90DF90CF90BF9054
S1131DB0AF909F908F900895CF93DF938AE00E9415
S1131DC0F10E809114078A3049F0C3E1D7E02196DF
S1131DD088810E94F10E89818A30C9F7DF91CF9101
S1131DE00895CF93C82F8A3019F48DE00E94F10E24
S1131DF05D9BFECFCCB9CF910895282FDB018FB71F
S1131E00F894382F90E08C918F3F69F0821759F045
S1131E109F5F943140F4FD01E90FF11DE081EF3F34
S1131E2011F0E217A9F7943199F0FD01E90FF11DC2
S1131E308081821769F4933140F4FD01E90FF11DAB
S1131E40818180839F5F9331C0F38FEF53968C938E
S1131E503FBF0895EF92FF920F931F93CF938FB7D5
S1131E60F894082FE091F504EE2309F06EC038E6EB
S1131E70E32E38E0F32E8091000180936808CE2F82
S1131E80F70132968FEF8193CF5FC431D8F3C0E06E
S1131E90809175058F3F99F0EC2FFF27DF01AB5838
S1131EA0BA4F8C91E859F74F8283CF5FC43138F42D
S1131EB0EC2FFF27EB58FA4F80818F3F69F7C4312D
S1131EC0B1F41FB71078F8948CE491E09F938F934A
S1131ED084E197E09F938F930E94080E0E94DC0E8A
S1131EE00F900F900F900F90112309F07894F70141
S1131EF0C18390E0C431D8F480913E088F3FB9F09B
S1131F00EC2FFF27E859F74FA92FBB27A25CB74F47
S1131F108C9182839F5FCF5F943148F4C43138F44D
S1131F20E92FFF27E25CF74F80818F3F49F723E6D3
S1131F3038E046E16FEF7FEF8FE10E94BA0F9927F7
S1131F40813019F48093F5040EC00E947C0864EF7C
S1131F5071E00E94D22FAA27BB279C01AD0161E04A
S1131F60862F0E94FA070FBFCF911F910F91FF9008
S1131F70EF900895CF92DF92EF92FF920F931F9309
S1131F80CF93DF93D82E7B01042FE90110915308DE
S1131F90112331F541E0C42EC09253080E3130F4C0
S1131FA08DEA97E20E94B302882319F41093530830
S1131FB017C0D093F904C093F8040C83E882F98223
S1131FC0DA82E091F804F091F904809102018383AC
S1131FD08C2D8E5F8C5F8B32E8F381E090E002C041
S1131FE080E090E0DF91CF911F910F91FF90EF90EF
S1131FF0DF90CF900895CF93C1E020E08FB7F8949D
S1132000382F809126088823C9F580918E08992756
S113201081FF09C088EB96E090936A058093690577
S113202080E490E01EC082FF12C0E0919204F0911F
S11320309304F0936A05E093690582E490E0909339
S11320409D0480939C0484819927059610C083FF86
S113205015C08BEC94E090936A05809369058FEF2B
S113206090E090939D0480939C0481E090E0909391
S1132070D6048093D5042C2FC09326083FBF222377
S1132080F1F08FB7F894992710923B0410923A0418
S113209010924306109242068FBF8EE70E9463108F
S11320A0C82F813061F08FB7F894282F332788E048
S11320B0809326082FBF8CE790E10E94B3028C2FF7
S11320C09927CF910895482F8FB7F894282F332755
S11320D090915F0681E080935F062FBF992319F0EA
S11320E080E090E008958FB7F89499274CB95E9AF0
S11320F08FBF81E090E0089561E08FB7F894282FB6
S1132100332780912608883019F460E0609326080C
S11321102FBF80919C0490919D0440918E0880343F
S1132120910551F48FB7F894282F332782E048277C
S113213040938E082FBF17C08FB7F894282F3327EA
S113214084E0482740938E082FBF80919204909199
S113215093040E94B6108FB7F894992710929304B1
S1132160109292048FBF0E94FB0F0895CF93DF93C8
S1132170FC0110925308828199278232910509F457
S11321808EC08332910554F48032910569F1813215
S113219091050CF056C04F9789F0E5C08432910543
S11321A009F49FC0843291050CF48AC085329105EC
S11321B009F4A9C0869709F4B5C0D5C08FB7F894BF
S11321C0C82F8091F504882309F4CCC01092F5043B
S11321D080918B05882309F0C5C00E947C0864EFB8
S11321E071E00E94D22F58C08FB7F894C82F809105
S11321F0F504882309F4B6C01092F5046623B9F0F7
S113220080913504882331F0809193088F5F809307
S1132210930803C081E0809335048091C3068F5FE7
S11322208093C30680915E088F5F80935E087091EF
S11322308B05713009F096C0809138089091390867
S11322402BC08FB7F894C82F8091F5048823D9F058
S11322501092F5046623B9F080911007882331F0B9
S1132260809110068F5F8093100603C081E08093F5
S113227010078091E2048F5F8093E204809134041C
S11322808F5F8093340480918B05823009F06AC09B
S11322908091BA059091BB05AA27BB275DC08FB773
S11322A0F894982F8091F504882359F11092F5043D
S11322B0613039F58091BE068F5F8093BE0621C0E0
S11322C08FB7F894982F8091F5048823D1F0109259
S11322D0F5046130B1F48091FA048F5F8093FA04BD
S11322E010C08FB7F894982F8091F504882349F093
S11322F01092F504613029F4809146068F5F809333
S113230046069FBF30C08FB7F894C82FDD27809151
S1132310F504882311F01092F50480918B05853023
S113232009F50EC08FB7F894C82FDD278091F50406
S1132330882311F01092F50480918B05863091F476
S11323400E947C0864E670E00E94D22FAA27BB2773
S113235088519C4FAF4FBF4F9C01AD0161E081E0BC
S11323600E94FA07CFBF81E090E0DF91CF910895FA
S11323701F93CF93FC0111E090E08FB7F894C82F1E
S113238080919E04882311F0192F2BC010939E0472
S1132390F0931207E093110784819927059690938F
S11323A0F7048093F60480911605882399F08091B0
S11323B09F04882331F40E9442128F719070019619
S11323C004C080E090E00E9465129093B10680936F
S11323D0B00604C01092B1061092B00681E080935A
S11323E0B3049091D004CFBF112309F446C09830B0
S11323F009F043C08FB7F894282F332783E08093E4
S1132400D0042FBF85E00E94A1126BE380E00E94FC
S1132410440769E380E00E94440788EC90E00000F0
S11324200000000000000000000000000000019710
S113243018161906A4F30E94DB07BB98BA9880EC1F
S11324408DB9B8980E946A0880913D068F3128F0B2
S113245020E03AE040E050E004C020E830E040E012
S113246050E060E084E00E94FA0720E230E040E0BF
S113247050E061E085E00E94FA07812F9927CF910F
S11324801F9108958FB7F894482F55272091D206AD
S11324903091D306832F881F8827881F220F331F6C
S11324A0882321F08BE090E1282739272F5F3F4FC5
S11324B03093D3062093D2068091DC049091DD04FE
S11324C0282739274FBFC90108959C0160915906F7
S11324D070915A064091540650915506892B11F17A
S11324E08091D6069091D70601969093D706809353
S11324F0D6066417750719F428303105B0F464174B
S1132500750771F02830310558F4C90108968832EE
S11325109105B0F00E9442128F719070099608954F
S1132520C90108956417750731F40E944212877037
S11325309070019608950E9442128F7190700996CE
S11325400895CF93DF93883008F03EC041E050E017
S113255060E070E004C0440F551F661F771F8A9522
S1132560D2F7C0915408D0915508E0915608F091E3
S11325705708CE01DF0184239523A623B7230097B0
S1132580A105B10509F18FB7F894282F3327DB0192
S1132590CA0180959095A095B0958C239D23AE2378
S11325A0BF238093540890935508A0935608B09382
S11325B057082FBF0097A105B10519F481E0809356
S11325C0530681E090E002C080E090E0DF91CF917B
S11325D008951F93CF93482F282F3327809100010C
S11325E0909101012817390709F447C04F3F09F4B6
S11325F044C08FB7F894C82F80E0909160069F3F45
S113260091F0941781F08F5F843168F4E82FFF27ED
S1132610EE0FFF1FEE0FFF1FE05AF94FE081EF3F6F
S113262011F0E41781F78431B9F41FB71078F894E6
S11326308DE291E09F938F9384E197E09F938F9332
S11326400E94080E0E94DC0E0F900F900F900F90C6
S1132650112391F0789410C0E82FFF27EE0FFF1F8D
S1132660EE0FFF1FE05AF94F8081841729F0408351
S113267063838FEF81838283CFBFCF911F910895AE
S1132680982F8FB7F894382F20E0809160068F3F01
S113269091F0891781F02F5F243168F4E22FFF272E
S11326A0EE0FFF1FEE0FFF1FE05AF94FE081EF3FDF
S11326B011F0E91781F7243131F1E22FFF27EE0FF2
S11326C0FF1FEE0FFF1FE05AF94F80818917D9F4DD
S11326D083818623C1F0233198F4E22FFF27EE0F84
S11326E0FF1FEE0FFF1FE05AF94F84819581A681E9
S11326F0B78180839183A283B3832F5F233168F3EF
S11327008FEF8093AC063FBF0895482F8F3F19F495
S113271024C0C901089590E0809160068F3FE9F0DC
S1132720292F3327F901EE0FFF1FEE0FFF1FE05A89
S1132730F94F8081841719F48381862351F79F5FB1
S1132740943158F4E92FFF27EE0FFF1FEE0FFF1F00
S1132750E05AF94F80818F3F19F78FEF9FEF08956B
S1132760CF93982F8FB7F894C82F8091F5048823BE
S1132770F9F4809100018093680890936C0880912B
S11327808B05809369088091C50580936A088091C0
S1132790B60680936B0823E638E045E06FEF7FEFE1
S11327A082E20E94BA0F9927813011F48093F504D4
S11327B0CFBFCF910895FF920F931F93CF93DF93D1
S11327C0EC018C010B5F1F4F61E08D810E9485132A
S11327D08F5F9F4F09F45DC080918B05823009F0B3
S11327E058C09091C5058D81981709F052C08FB7D4
S11327F0F894F82E81E00E94A112F80164818D8181
S11328000E945014882361F1F80124819D818FB7BF
S1132810F894182F8091F504882309F5809100011C
S11328208093680890936D0820936C0880918B05C1
S1132830809369088091B60680936B088091C505E2
S113284080936A0823E638E046E06FEF7FEF84E286
S11328500E94BA0F9927813011F48093F5041FBFA9
S113286080914A06882321F084E080938B050BC075
S113287083E080938B0524E630E040E050E061E0A3
S113288082E00E94FA07109210078FEF8093C5052B
S1132890FFBECE01DF91CF911F910F91FF9008955C
S11328A0282F6F3F41F18F3F29F425C0618381E0D8
S11328B090E0089590E0809160068F3FE1F0E92F69
S11328C0FF27EE0FFF1FEE0FFF1FE05AF94F808125
S11328D0821719F481818F3F49F39F5F943158F433
S11328E0E92FFF27EE0FFF1FEE0FFF1FE05AF94FEE
S11328F080818F3F21F780E090E00895CF93DF93AC
S1132900FC01E41BF50B6217730710F0EF0102C022
S1132910EF012197DB01A21BB30BBD01CE01DF91B7
S1132920CF91089590E0492F809160068F3FE9F0A0
S1132930E42FFF27EE0FFF1FEE0FFF1FE05AF94FA2
S11329408381282F332720FF02C022FF9F5F4F5F20
S1132950443158F4E42FFF27EE0FFF1FEE0FFF1F43
S1132960E05AF94F80818F3F19F7892F99270895ED
S11329701F93CF938FB7F894C82F10E040E050E036
S113298060E070E0809160068F3F41F1E12FFF2706
S1132990EE0FFF1FEE0FFF1FE05AF94F21812F3F6B
S11329A079F081E090E002C0880F991F2A95E2F740
S11329B0AA2797FDA095BA2F482B592B6A2B7B2B5E
S11329C01F5F143158F4E12FFF27EE0FFF1FEE0FA6
S11329D0FF1FE05AF94F80818F3FC1F610E020E0DD
S11329E030E081E090E0022E02C0880F991F0A9423
S11329F0E2F7AA2797FDA095BA2F84239523A6234F
S1132A00B7230097A105B10501F11F5F2F5F3F4F69
S1132A10103238F380914A068823E9F41FB71078FE
S1132A20F8948AE791E09F938F9384E197E09F93D2
S1132A308F930E94080E0E94DC0E0F900F900F904F
S1132A400F90112391F0789410C01093A60481E0A4
S1132A5080934A06DFCF84E080938B058091A6049F
S1132A600E94B01381E00E94A112CFBFCF911F91A9
S1132A700895CF92DF92EF92FF920F931F93CF931B
S1132A80DF9380E398E00E94B6078091C60490919A
S1132A90C704A091C804B091C904E0903008F09034
S1132AA0310800913208109133089C01AD01C8012E
S1132AB0B7010E947E14DC01CB018093A0049093A3
S1132AC0A104A093A204B093A3048091D104909193
S1132AD0D204A091D304B091D4049C01AD01C801E7
S1132AE0B7010E947E146B017C011FB71078F89423
S1132AF08091A0049091A1049F938F938091A2044C
S1132B009091A3049F938F938091100699279F938C
S1132B108F938091930899279F938F939091C306E5
S1132B208091E204890F912D911D2091FA04820F66
S1132B30911D2091BE06820F911D20914606820FA1
S1132B40911D9F938F9380910001909101019F9318
S1132B508F9383EB91E09F938F93C4E1D7E0DF934E
S1132B60CF930E94080E0E94DC0E8DB79EB740964C
S1132B700FB6F8949EBF0FBE8DBF112309F0789451
S1132B801FB71078F8948091460699279F938F93E6
S1132B908091BE0699279F938F938091FA04992779
S1132BA09F938F938091E20499279F938F938091B1
S1132BB0C30699279F938F938091000190910101FF
S1132BC09F938F938CEE91E09F938F93DF93CF939A
S1132BD00E94080E0E94DC0E8DB79EB740960FB679
S1132BE0F8949EBF0FBE8DBF112309F078941FB7D0
S1132BF01078F894DF92CF92FF92EF928091A6041E
S1132C0099279F938F938091B60699279F938F93CB
S1132C1080910001909101019F938F9389E292E04A
S1132C209F938F93DF93CF930E94080E0E94DC0E34
S1132C308DB79EB70E960FB6F8949EBF0FBE8DBF8C
S1132C40112309F07894DF91CF911F910F91FF9098
S1132C50EF90DF90CF900895EF92FF921F93CF9360
S1132C601FB71078F89421E6E22E22E0F22EFF92AC
S1132C70EF9284E197E09F938F930E94080E0E9445
S1132C80DC0E0F900F900F900F90112309F07894A1
S1132C90C0E0809160068F3F09F4CAC080918B0523
S1132CA099278430910509F43CC0853091051CF4C2
S1132CB0039729F0AEC0069709F465C0AAC0EC2FAB
S1132CC0FF27EE0FFF1FEE0FFF1FE05AF94F83811E
S1132CD0992780FF12C01FB71078F8948281992732
S1132CE09F938F93818199279F938F9380819927B5
S1132CF09F938F938AE992E077C081FF8AC01FB7C0
S1132D001078F894828199279F938F9381819927D2
S1132D109F938F93808199279F938F938CEB92E05D
S1132D2063C0EC2FFF27EE0FFF1FEE0FFF1FE05ACB
S1132D30F94F8381992780FF12C01FB71078F89448
S1132D40828199279F938F93818199279F938F9352
S1132D50808199279F938F938EED92E045C081FFE8
S1132D6058C01FB71078F894828199279F938F9346
S1132D70818199279F938F93808199279F938F9324
S1132D8080E093E031C0EC2FFF27EE0FFF1FEE0F22
S1132D90FF1FE05AF94F8381992780FF12C01FB7A4
S1132DA01078F894828199279F938F938181992732
S1132DB09F938F93808199279F938F9382E293E0CF
S1132DC013C081FF26C01FB71078F8948281992719
S1132DD09F938F93818199279F938F9380819927C4
S1132DE09F938F9384E493E09F938F9384E197E080
S1132DF09F938F930E94080E0E94DC0E8DB79EB79E
S1132E000A960FB6F8949EBF0FBE8DBF112309F02A
S1132E107894CF5FC43160F4EC2FFF27EE0FFF1FCF
S1132E20EE0FFF1FE05AF94F80818F3F09F036CF34
S1132E301FB71078F894FF92EF9284E197E09F9384
S1132E408F930E94080E0E94DC0E0F900F900F903B
S1132E500F90112309F07894CF911F91FF90EF9078
S1132E6008958091CA048F3130F00E94671706C01C
S1132E7081E090E023C08F5F8093CA0490E080914A
S1132E8060068F3FC9F0E92FFF27EE0FFF1FEE0FFB
S1132E90FF1FE05AF94F81818F3F51F39F5F9431B7
S1132EA058F4E92FFF27EE0FFF1FEE0FFF1FE05A24
S1132EB0F94F80818F3F39F780E090E0882319F43F
S1132EC00E949D17089580E00E94FF1708951F93A4
S1132ED0CF93DF93CCEAD6E098819F3F29F1898193
S1132EE08F3F11F51FB71078F894892F99279F9376
S1132EF08F9386E693E09F938F9384E197E09F936B
S1132F008F930E94080E0E94DC0E8DB79EB7069622
S1132F100FB6F8949EBF0FBE8DBF112309F07894AD
S1132F206B8188810E944013249796E0C036D907AC
S1132F309CF6DF91CF911F9108951F930E9467170C
S1132F4081E00E94A1120E94DB1720E0882321F077
S1132F5086952F5F8823E1F781E090E002C0880F17
S1132F60991F2A95E2F78093A7041FB71078F89465
S1132F700E94DB1799279F938F938091A704992729
S1132F809F938F938DE893E09F938F9384E197E0D1
S1132F909F938F930E94080E0E94DC0E8DB79EB7FC
S1132FA008960FB6F8949EBF0FBE8DBF112309F08B
S1132FB078941F9108959091A60420E08091600672
S1132FC08F3FD1F0E22FFF27EE0FFF1FEE0FFF1F01
S1132FD0E05AF94F8181981708F4982F2F5F243114
S1132FE058F4E22FFF27EE0FFF1FEE0FFF1FE05AEA
S1132FF0F94F80818F3F31F7892F992708951F93C7
S1133000CF93DF93982F8FB7F894182FE091F5049E
S1133010EE2309F04EC02091A60420936908309154
S113302000013093680890936A089E2FEBE6F8E05D
S11330308FEF81939F5F9431D8F390E08091600685
S11330408F3F01F1A92FBB27AA0FBB1FAA0FBB1FDC
S1133050A05AB94F1196EC911197EF3F29F0FF2731
S1133060E559F74F8C9180839F5F943158F4E92F91
S1133070FF27EE0FFF1FEE0FFF1FE05AF94F80816D
S11330808F3F01F780914A06882329F0E22FFF271A
S1133090E559F74F308323E638E047E16FEF7FEFE0
S11330A085E20E94BA0F9927813019F48093F504C0
S11330B012C00E947C0864E670E00E94D22FAA2706
S11330C0BB2788519C4FAF4FBF4F9C01AD0161E0BE
S11330D0862F0E94FA071FBFDF91CF911F91089599
S11330E01F93CF93DF93809136048F3198F1CCEA0C
S11330F0D6E098819F3F29F18A818F3F11F51FB750
S11331001078F894892F99279F938F9385EB93E0F8
S11331109F938F9384E197E09F938F930E94080E6F
S11331208DB79EB706960FB6F8949EBF0FBE8DBF9F
S11331300E94DC0E112309F078946B8188810E942F
S11331404013249796E0C036D9079CF606C081E068
S113315090E023C08F5F8093360490E080916006F6
S11331608F3FC9F0E92FFF27EE0FFF1FEE0FFF1F60
S1133170E05AF94F82818F3F51F39F5F943158F4A5
S1133180E92FFF27EE0FFF1FEE0FFF1FE05AF94F45
S113319080818F3F39F780E090E0882369F481E0F3
S11331A00E94A11280916B05882349F481E08093E9
S11331B06B050E942C1603C082E00E94E318DF9185
S11331C0CF911F910895CF93982F8FB7F894C82F5C
S11331D0E091F504EE2309F050C080910001809342
S11331E068088091A7048093690890936A089E2FC9
S11331F0E8E6F8E08FEF8383828B9F5F31969F3000
S1133200C8F390E0392F809160068F3F41F1A92FD8
S1133210BB27AA0FBB1FAA0FBB1FA05AB94F1396F7
S11332208C91139780FF0DC012962C9112972F3F0B
S113323041F0E32FFF27E859F74F8C918383228BCA
S11332403F5F9F5F943158F4E92FFF27EE0FFF1F74
S1133250EE0FFF1FE05AF94F80818F3FC1F623E63E
S113326038E041E26FEF7FEF86E20E94BA0F9927C0
S1133270813019F48093F50412C00E947C0864E63E
S113328070E00E94D22FAA27BB2788519C4FAF4FD2
S1133290BF4F9C01AD0161E0862F0E94FA07CFBFAA
S11332A0CF9108951F920F920FB60F921124CF92CF
S11332B0DF92EF92FF920F931F932F933F934F93BD
S11332C05F936F937F938F939F93AF93BF93CF93AA
S11332D0DF93EF93FF93C4B1D5B1D370349A379889
S11332E07894EFEF00E011E08091730590917405FC
S11332F00A9759F4CE01AA27BB27809358089093C4
S11333005908A0935A08B0935B088FB7F894F82F24
S1133310D0907305ED2CFF2461E070E00E2C02C008
S1133320660F771F0A94E2F7409191085091920832
S1133330462357234115510551F48091C6059091B8
S1133340C705862797279093C7058093C6052091C4
S11333504F0630915006CB0182239323892B49F0E9
S1133360012F452B31F4262737273093500620931D
S11333704F064091C6055091C7054115510501F10D
S113338020917305309174052F5F3F4F2C30310528
S113339011F0C90102C080E090E09C0181E090E05E
S11333A0022E02C0880F991F0A94E2F78423952302
S11333B0892B51F33093740520937305E0917305C1
S11333C0FFBFEF3F19F08E2F0E94401B8AE0D816F2
S11333D009F421C1002311F010E01DC1E114F1042E
S11333E009F017C18FB7F894C82E2091D004822F0A
S11333F099278430910529F1853091051CF40397B0
S113340041F004C18630910591F0099709F47CC01C
S1133410FDC08091DA04833009F04CC0D093480594
S1133420C093470582E59BE10E94B30243C08091AB
S1133430DA04863009F03EC0D093B306C093B206D6
S113344039C0809160088F5F809360088091B705D0
S11334509091B80540968C179D0720F08091160531
S1133460882359F58091DA04843039F51AEA8FB744
S1133470F8949927109349058FBF0E94FB1BBB9AB0
S1133480BA9AD093B306C093B20685E080936008DD
S113349081E08093D806F0922B08E0922A08F092FB
S11334A01B05E0921A058093D00482E080933704D0
S11334B01093E0060093DA04A9C01092DA04809114
S11334C060088530B1F48091D6069091D7060196B4
S11334D09093D7068093D6060E9442128F70907004
S11334E001969093B1068093B00683E08093D00454
S11334F08DC02093DA048FB7F894082F112780E049
S11335000E942A1C0FBF82C0F02E8091B7059091B3
S1133510B8059C013695279536952795821B930B04
S11335208C179D0748F4D0934805C093470582E55E
S11335309BE10E94B30249C08091A404863098F0B4
S11335400E94DB0783E08093D004BB98BA9880EC98
S11335508DB9B8980E946A088CE59CE10E94B30278
S113356051E0F52E32C00E94DB078FB7F894082F84
S113357011278F2D0E942A1C0FBF8823A9F080E5F4
S113358090E00000000000000000000000000000C7
S11335900000019718161906A4F38091A4048F5F04
S11335A08093A40441E0F42E80914B0690914C0644
S11335B0019690934C0680934B066FE380E00E9443
S11335C0440760E08BE00E9444078091B3048823A1
S11335D091F00E94DB0783E08093D004BB98BA98F3
S11335E080EC8DB9B8980E946A088CE59CE10E9431
S11335F0B30231E0F32EFF2049F488E698E20E94FA
S1133600B30288E08093D0040E94761CCFBE81E090
S113361001C080E0182F8FB7F894682F41E050E084
S113362002C0440F551FDA94E2F7209191083091BB
S11336309208C90184239523892B41F0112331F485
S11336402427352730939208209391086FBFFF9168
S1133650EF91DF91CF91BF91AF919F918F917F9126
S11336606F915F914F913F912F911F910F91FF9017
S1133670EF90DF90CF900F900FBE0F901F90189592
S1133680982F8FB7F894282F3327E5E1F8E0E90F56
S1133690F11D80818F7187B92FBF379A369A81E0E7
S11336A090E008950F931F93CF93DF93CDB7DEB7C8
S11336B062970FB6F894DEBF0FBECDBF8FB7F894F4
S11336C0482F552720911505E22FFF27EE0FFF1FE6
S11336D0EC54FB4F8091470590914805808391837A
S11336E0822F8F5F80931505893010F01092150595
S11336F080913D068F3118F48F5F80933D064FBF54
S113370048E0A4EBB4E020E030E0FE01E20FF31F58
S11337108D919D918183928341502E5F3F4F47FF4E
S1133720F4CF50E0A52F41E022E030E0BE016F5F0E
S11337307F4FF901E60FF71F80819181EFEF8F3FF3
S11337409E0791F0EA2FFF27E7FDF095EE0FFF1F8C
S1133750E60FF71F0190F081E02DE817F90718F044
S1133760EF5FFF4F09F4A42F4F5F2E5F3F4F4930A7
S1133770ECF2EA2FFF27E7FDF095EE0FFF1FE60FAF
S1133780F71F608171818FEF9FEF808391835F5F6B
S113379053304CF28091B7059091B805F5E0880F4D
S11337A0991FFA95E1F79C0144275527660F771F67
S11337B0CB01AA27BB27280F391F4A1F5B1F8FB7CE
S11337C0F894082F1127CA01B90122E230E040E041
S11337D050E00E94E62F3093B8052093B7050FBF41
S11337E062960FB6F894DEBF0FBECDBFDF91CF91C6
S11337F01F910F91089561EE80E00E94440780912B
S11338006705682F89E00E9444078AEF90E0000072
S1133810000000000000000000000000000001970C
S113382018161906A4F380915505682F8BE00E94A1
S1133830440784E190E00000000000000000000064
S1133840000000000000019718161906A4F381E097
S113385090E00895CF93DF93782F41E050E061E04A
S1133860C82FDD270C2E02C0440F551F0A94E2F71F
S11338702091C6053091C705CA0182239323892B61
S113388011F060E014C0CA01822B932B9093C705FA
S11338908093C605232B59F4872F0E94401B992738
S11338A0682F882321F0D0937405C0937305862F65
S11338B09927DF91CF91089580913D068F3128F0AB
S11338C020E03AE040E050E004C020E830E040E08E
S11338D050E060E084E00E94FA072EE130E040E02E
S11338E050E061E085E00E94FA0708956F98B89A65
S11338F0C0980E946A0881E090E0089578941F922D
S11339000F920FB60F9211242F933F934F935F930F
S11339106F937F938F939F93AF93BF93CF93DF93D3
S1133920EF93FF938FB7F894282F33278091FD04EA
S1133930882369F0809147068093DD068860809330
S1133940470683BF8091120581BF1092FD042FBFEB
S11339508FB7F894C82FDD278091480690914906C7
S1133960892B21F485E798E20E94B30221B7809164
S1133970480690914906820F911D0196909349063D
S113398080934806CFBFFF91EF91DF91CF91BF9114
S1133990AF919F918F917F916F915F914F913F91E3
S11339A02F910F900FBE0F901F90189590E0292F24
S11339B0809160068F3FD1F0E22FFF27EE0FFF1FAB
S11339C0EE0FFF1FE05AF94F81818F3F09F49F5F8B
S11339D02F5F243158F4E22FFF27EE0FFF1FEE0F65
S11339E0FF1FE05AF94F80818F3F31F79F5F892F86
S11339F099270895FF920F931F93CF938FB7F8944D
S1133A00F82EC091F504CC2309F064C008E618E050
S1133A108091000180936808C80107960E94B60748
S1133A2080918B05809369088091B60680936B081A
S1133A308091C50580936A082C2F3C2F80916006E5
S1133A408F3F29F1A32FBB27AA0FBB1FAA0FBB1FB0
S1133A50A05AB94F13968C911397992780FF09C0E8
S1133A6082FD07C0E22FFF27ED58F74F8C9180832A
S1133A702F5F3F5F343158F4E32FFF27EE0FFF1F12
S1133A80EE0FFF1FE05AF94F80818F3FD9F62431A2
S1133A9048F4E22FFF27ED58F74F8FEF80832F5F15
S1133AA02431B8F30E949214F8018483809197041E
S1133AB0909198048583968323E638E04FE16FEF75
S1133AC07FEF80E20E94BA0F9927813019F4809326
S1133AD0F5040CC08091380890913908AA27BB27B7
S1133AE09C01AD0161E0862F0E94FA07FFBECF91D1
S1133AF01F910F91FF9008958F929F92AF92BF9262
S1133B00CF92DF92EF92FF920F931F93CF93DF93A5
S1133B10CDB7DEB72C970FB6F894DEBF0FBECDBF7E
S1133B20682F80912708811160958091D00499278E
S1133B308430910509F46BC2853091055CF48230C0
S1133B40910509F4D7C4833091050CF0E0C10197C5
S1133B5069F0D0C48630910509F4D5C28630910548
S1133B600CF479C2079709F474C4C4C42091E00624
S1133B708FB7F8949927209349058FBF40912A085D
S1133B8050912B084F5F5F4F50932B0840932A08A6
S1133B908091370499278530910509F4F5C0863062
S1133BA0910554F483309105B1F1843091050CF002
S1133BB06AC0029769F087C18730910509F422C170
S1133BC0873091050CF4F9C0089709F445C17BC10D
S1133BD08091E7049091E80401969093E80480931F
S1133BE0E7048091E9049091EA044817590770F4B6
S1133BF0E0911107F091120784A195A18F5F9F4F67
S1133C0009F078C44830510508F474C483E3809300
S1133C10E00683E055C18091E7049091E8040196A1
S1133C209093E8048093E7048CEC8093E00684E0AE
S1133C30809337048FEF9FEF90932B0880932A088B
S1133C40E0901107F0901207F70182818F3D09F08F
S1133C5051C487010B5F1F4FCE0101960E94B60726
S1133C608B819C81F7018583968389819A81F801F0
S1133C708283938381E08483809100019091010188
S1133C808583968337C48091E7049091E804019674
S1133C909093E8048093E70480912A08282F33271F
S1133CA08091F6049091F7042817390708F066C04C
S1133CB0E0911107F091120782818F3DE1F54530C3
S1133CC05105C9F555E0E52EF12CEE0EFF1E6E01EF
S1133CD00894C11CD11CC6010E94B6078091EB0454
S1133CE09091EC0429813A81B901680F791F4B81C5
S1133CF05C81E091ED04F091EE048095909582173B
S1133D00930748F46F5F7F4F69837A834E0F5F1F79
S1133D104F5F5F4F04C069837A834E0F5F1F4B83ED
S1133D205C83F60182819381F70180839183898189
S1133D309A8182839383E0911107F0911207809115
S1133D402A0890912B08E80FF91F20812093E006A0
S1133D5080911A0590911B05EAE6F1E02927220FCC
S1133D60F11DE20FF11DC895982F802D3196C8954D
S1133D70902590931B0580931A05BCC380911A0566
S1133D808093E00685E09CC08091E7049091E8046C
S1133D9001969093E8048093E70480911A0590912A
S1133DA01B05892F99278093E00686E080933704CA
S1133DB010922B0810922A089DC38091E7049091D9
S1133DC0E80401969093E8048093E7044430510595
S1133DD008F490C310922B0810922A0880913C0694
S1133DE0882311F087E06CC080916F059091700575
S1133DF001969093700580936F05BB98BA980E94C2
S1133E00DB075DC04130510571F48091E704909166
S1133E10E80401969093E8048093E704BB98BA9869
S1133E200E94DB0767C380913A0890913B08019692
S1133E3090933B0880933A084430510508F45AC3E0
S1133E4088E08093370410922B0810922A0810926D
S1133E509508109294084EC380913A0890913B08BB
S1133E60019690933B0880933A0820E0809194084F
S1133E7090919508880F991F9093950880939408C2
S1133E8067FF05C081609093950880939408660F3E
S1133E90809194089091950883589A4B09F414C31F
S1133EA02F5F283018F380912A0890912B084297AD
S1133EB008F420C3E0911107F091120716A289E0DB
S1133EC08093370417C31092B304E0911107F09163
S1133ED0120782818E5D823020F4809114088093D1
S1133EE03C0683EF97E20E94B302882309F402C3DD
S1133EF023E02093D00480914406909145060196D6
S1133F0090934506809344062093DA0499C28091E5
S1133F103A0890913B08019690933B0880933A08A5
S1133F206A3A11F0653521F580915C0890915D083D
S1133F30019690935D0880935C08039708F4DAC2B5
S1133F401092520810925D0810925C0810926E054F
S1133F5010926D051092FB0410921B0510921A0525
S1133F6082E290E090933F0680933E0685E070C025
S1133F7080919F04882359F180914D06882339F15B
S1133F8081E090E0A0E0B0E00090590604C0880F02
S1133F90991FAA1FBB1F0A94D2F72FB7F894622F58
S1133FA02091C1053091C2054091C3055091C405CB
S1133FB082239323A423B5230097A105B10511F00F
S1133FC081E001C080E06FBF882309F093C2809133
S1133FD0B304882309F48EC28091B0069091B1068F
S1133FE001979093B1068093B006181619060CF445
S1133FF081C284E08093D0048093DA041092D806BE
S11340001092600810925D0810925C0819C28091A9
S11340103A0890913B08019690933B0880933A08A4
S11340206A3A19F0653509F065C28091D606909117
S1134030D70601969093D7068093D6060E94421223
S11340408F70907001969093B1068093B00683E0D0
S11340508093D0044FC280913A0890913B08019616
S113406090933B0880933A086A3A11F0653519F445
S1134070609314053FC2809152089927009719F064
S11340800697C4F503C06093130537C02091130548
S113409030911405922F882790931405809313056B
S11340A060931305FF24220F331F67FD2160660F01
S11340B083E32C3C3807C9F4E0915106F091520691
S11340C094819923B9F486E08093D0048093DA0430
S11340D08FB7F894082F1127892F0E942A1C0FBF2D
S11340E087E08F198093FB0408C0F394E7E0EF1591
S11340F0D0F603C083E08093D004809152088F5F90
S113410080935208F7C180913A0890913B08019638
S113411090933B0880933A0880911305909114057D
S1134120982F8827909314058093130560931305A3
S113413020911305309114050090FB0402C03695BC
S113414027950A94E2F7F22EE0915106F091520677
S113415080916D0590916E05E80FF91F20834091C1
S11341606D0550916E054F5F5F4F50936E05409300
S11341706D0580913E0690913F064817590788F5D2
S113418080911A0590911B05EAE6F1E0F926FF0CEF
S1134190F11DEF0DF11DC895982F802D3196C8950E
S11341A0902590931B0580931A054530510509F01D
S11341B0A1C1E0915106F091520684819927909310
S11341C03F0680933E068E31910528F0148283E0E9
S11341D08093D004ECC1059690933F0680933E06ED
S11341E089C14817590709F0B0C0A0915106B09190
S11341F05206FD0112968C9112978F3D09F089C0E9
S11342008FB7F894E82E9D012B5F3F4FB5E08B2EBE
S1134210912C8C0E9D1E858196818F839887F90140
S1134220828193818D839E838481C82EDD24858140
S1134230968190939A0480939904A9E0AA2EB12CB4
S1134240AC0EBD1EC5010E94B6072F8138858B8533
S11342509C858217930750F02817390760F02D8149
S11342603E8189859A858217930710F401E006C080
S11342702817390710F402E001C003E0013019F4F3
S1134280A501B40104C0023039F4A401B50189EDDB
S113429096E00E94EC2208C01092DA061092D90629
S11342A0E9EDF6E0128213820093C006C114D10432
S11342B019F4F1E0CF2ED12CF8E0CF16D10440F55B
S11342C060E070E06C157D0518F52091DB063091F7
S11342D0DC068091D9069091DA06A9015695479596
S11342E06F5F7F4F20FF06C09A0196958795815096
S11342F0904803C09A01969587956C157D0568F3DF
S11343009093DA068093D9063093DC062093DB067B
S1134310EFBE80911A0590911B05EAE6F1E0F926BB
S1134320FF0CF11DEF0DF11DC895982F802D3196CE
S1134330C895902590931B0580931A0582E290E01E
S113434090936E0580936D05D5C04432510508F4F1
S1134350D1C0E0915106F091520622A133A180917F
S11343601A0590911B052817390781F582818F3D25
S113437021F489ED97E20E94B302E0915106F09195
S1134380520681E090E082A393A380913C068823A7
S1134390F9F0208131818091000190910101281769
S11343A03907B1F487E08093D0040E94FB1BBB9AC9
S11343B0BA9A8FB7F894282F33278AEA809349054D
S11343C02FBF10926E0510926D05F1C012A213A2B8
S11343D00E94761C83E08093D00480919F048130F6
S11343E071F48091B304882351F08091B0069091C8
S11343F0B1060E9465129093B1068093B006E091D5
S11344005106F09152068091B2069091B30684A3AE
S113441095A385E193E20E94B302882369F4E091B5
S11344205106F0915206848383E08093D00480EC9B
S11344308DB9B8980E946A088091D0048093DA04F8
S11344408FB7F894082F112780E00E942A1C0FBF11
S113445051C08091E7049091E80401969093E80498
S11344608093E704E0916D05F0916E053196F09329
S11344706E05E0936D05E031F10580F10E94DB07E4
S1134480BB98BA980E94761C03E00093D004E09194
S11344905106F09152068091B2069091B30684A31E
S11344A095A385E193E20E94B302882319F5E09174
S11344B05106F091520684830093D00480EC8DB9A8
S11344C0B8980E946A0816C0E0911107F09112078B
S11344D081E086A389E08093370469C0EB30F1055D
S11344E048F0E850FF4F20818FB7F8949927209324
S11344F049058FBF20914B0630914C062536310576
S1134500C0F08091D0069091D10601969093D10687
S11345108093D0068091950490919604019690938F
S11345209604809395042456304030934C0620938F
S11345304B062091E7043091E80425363105C0F09C
S11345408091D0069091D10601969093D1068093E4
S1134550D00680915706909158060196909358067C
S113456080935706245630403093E8042093E704A0
S113457020913A0830913B0825363105C0F08091EE
S1134580D0069091D10601969093D1068093D006DF
S113459080917105909172050196909372058093B4
S11345A071052456304030933B0820933A0881E04B
S11345B090E02C960FB6F894DEBF0FBECDBFDF910E
S11345C0CF911F910F91FF90EF90DF90CF90BF900C
S11345D0AF909F908F900895CF93DF93EC01FB01F0
S11345E0DA018D919C91119720813181428153810F
S11345F012966D917C9113972817390758F4821BF2
S1134600930B8095909588839983461B570B415053
S1134610504006C0281B390B28833983461B570B8F
S11346204A835B83DF91CF9108951F93CF93DF93E8
S11346308FB7F894182F80914406909145068536DB
S1134640910570F080913C068093140810923C060A
S11346508CE195E00E94B811109245061092440630
S11346608091440690914506019690934506809367
S113467044062091510630915206F90117A210A662
S1134680E901D901159660919F04613009F05FC07A
S11346908091E104882309F45AC082818E3D09F097
S11346A056C082A193A1892B09F451C013968D9110
S11346B09C91149740910001509101018417950732
S11346C009F445C08D81882339F511962D913C91CB
S11346D012972417350701F56093EA0680915B066B
S11346E090915C069093EC068093EB063093EE0673
S11346F02093ED0690919E04992359F480913C06F1
S11347008093140890933C0685EE96E00E94B811BD
S113471027C06093B90524C08C91813009F580933A
S11347204D0613962D913C91149780915B069091C0
S11347305C0628173907A1F4109236081092250850
S113474010922408109239041092380409C0F90117
S113475082818E5D823020F0C9010E949F08EC01A5
S1134760209721F0D0935206C0935106E091510650
S1134770F091520614821FBF80EC8DB9B8980E9444
S11347806A08DF91CF911F91089578941F920F9238
S11347900FB60F9211246F927F928F929F92AF92D5
S11347A0BF92CF92DF92EF92FF920F931F932F93BA
S11347B03F934F935F936F937F938F939F93AF93A5
S11347C0BF93EF93FF93CF93DF93CDB7DEB72497D7
S11347D0F894DEBF7894CDBF8091E304882309F474
S11347E0F4C08091BD068230A9F48091E1069091D5
S11347F0E20680959095909389008093880080913B
S1134800B1049091B2042091E3063091E406821B36
S1134810930B15C08130B9F48091E1069091E206C2
S113482090938900809388008091B1049091B204A0
S11348302091E3063091E406820F931F0196909332
S1134840B2048093B1041092E3048091E0048823BD
S113485009F4C4C0CE0101960E94B6070B811C81E5
S1134860C801AA2797FDA095BA2FBC01CD010E94CB
S1134870092F17FF06C020E030E040E857E40E940B
S11348805C2E25EE38E34EE054E40E94782F6B0151
S11348907C0109811A81C801AA2797FDA095BA2F26
S11348A0BC01CD010E94092F17FF06C020E030E0B3
S11348B040E857E40E945C2E28EE38E34EE05CE3C7
S11348C00E94782FDC01CB019C01AD01C701B60128
S11348D00E945C2EDC01CB01BC01CD010E94EC2EB8
S11348E04B015C0160903408709035087301002717
S11348F01127A80197010E94E62FDC01CB01A80132
S11349009701281B390B4A0B5B0B57FD05C0CA01E5
S1134910B9010E94092F16C0DA01C9018170907093
S1134920A070B0705695479537952795822B932B99
S1134930A42BB52BBC01CD010E94092F9B01AC0116
S11349400E945C2E2FE632E143E85FE30E94782F59
S1134950DC01CB01BC01CD010E94EC2E6B017C017A
S1134960930144275527C501B4010E94E62F2093E3
S1134970B9063093BA064093BB065093BC068091A7
S1134980DE049091DF0401972091B9063091BA06B4
S11349908223932390935A06809359068091F104BD
S11349A09091F2040197282339233093F004209343
S11349B0EF0460919F04613029F4A701960186E019
S11349C00E94FA071092E00409C08091B10490910A
S11349D0B20401969093B2048093B1042496F8949F
S11349E0DEBFCDBFDF91CF91FF91EF91BF91AF912A
S11349F09F918F917F916F915F914F913F912F91F3
S1134A001F910F91FF90EF90DF90CF90BF90AF90E8
S1134A109F908F907F906F900F900FBE0F901F907C
S1134A201895382F8091230899278230910509F42D
S1134A306BC0833091052CF4009759F0019781F1F4
S1134A40B7C18330910509F49CC0049709F459C196
S1134A50AFC13E3709F0AEC18091B7069927FC017A
S1134A60EE0FFF1FEE0FFF1FE80FF91FE80FF91FEE
S1134A70EC53F94F82819381009709F09BC1118215
S1134A8090931805809317059093E6048093E504AA
S1134A90848195819093DF068093DE0681E085C151
S1134AA03E3709F487C18091B7069927FC01EE0FC0
S1134AB0FF1FEE0FFF1FE80FF91FE80FF91FEC535C
S1134AC0F94F30838091170590911805EAE6F1E0DB
S1134AD0232F2927220FF11DE20FF11DC895982FCE
S1134AE0802D3196C89590259093180580931705CD
S1134AF0832F99278134910529F08234910509F493
S1134B0053C156C182E051C13E3709F451C160918D
S1134B10B7063D3781F4862F9927FC01EE0FFF1F5E
S1134B20EE0FFF1FE80FF91FE80FF91FEC53F94FC1
S1134B3080E281833FC1862F9927FC01EE0FFF1F7E
S1134B40EE0FFF1FE80FF91FE80FF91FEC53F94FA1
S1134B502181232721838091170590911805EAE686
S1134B60F1E02927220FF11DE20FF11DC895982FBE
S1134B70802D3196C895902590931805809317053C
S1134B8013C14091E5045091E6044C32510508F0FC
S1134B90BAC03D3711F484E008C13E3709F07FC044
S1134BA04230510508F45FC0E091DE06F091DF0663
S1134BB0E40FF51F82919927382F22278291992794
S1134BC0282B392B80911705909118056091B70611
S1134BD028173907E1F4862F9927FC01EE0FFF1FF0
S1134BE0EE0FFF1FE80FF91FE80FF91FEC53F94F01
S1134BF0425050404283538383E899E20E94B302B7
S1134C008091B7068F5F81708093B70610C0862F9E
S1134C109927FC01EE0FFF1FEE0FFF1FE80FF91F8E
S1134C20E80FF91FEC53F94F12821382118280911D
S1134C30B7069927FC01EE0FFF1FEE0FFF1FE80FC9
S1134C40F91FE80FF91FEC53F94F82819381892BE7
S1134C50D9F4848195819093DF068093DE0681E008
S1134C608093230813C08091B7069927FC01EE0FA7
S1134C70FF1FEE0FFF1FE80FF91FE80FF91FEC539A
S1134C80F94F128213821182109223081092180590
S1134C90109217051092E6041092E5048BC0E0917F
S1134CA0DE06F091DF06E40FF51F30834091E50442
S1134CB05091E60442305105E8F0209117053091F7
S1134CC01805E091DE06F091DF06E40FF51F329738
S1134CD08081EAE6F1E08327880FF11DE80FF11DDA
S1134CE0C895322F202D3196C8953025309318055C
S1134CF0209317054F5F5F4F5093E6044093E504FC
S1134D0059C03E37D1F4109218051092170510922D
S1134D10E6041092E5048091B7069927FC01EE0F92
S1134D20FF1FEE0FFF1FE80FF91FE80FF91FEC53E9
S1134D30F94F1282138211823BC080E28327E091F3
S1134D40DE06F091DF062091E5043091E604E20FDF
S1134D50F31F80834091E5045091E60442305105ED
S1134D60E8F02091170530911805E091DE06F091E6
S1134D70DF06E40FF51F32978081EAE6F1E083272E
S1134D80880FF11DE80FF11DC895322F202D3196A3
S1134D90C895302530931805209317054F5F5F4F52
S1134DA05093E6044093E50483E08093230802C013
S1134DB01092230881E090E008958FB7F894992722
S1134DC020915F0610925F068FBF222309F4A4C0CE
S1134DD080912608873031F4109226088CE790E100
S1134DE00E94B30221E0809126089927843091051E
S1134DF009F46EC08530910554F48230910561F157
S1134E00833091050CF058C0019749F07CC086307E
S1134E10910509F471C006970CF463C074C082E074
S1134E208093260820913A0430913B0480919C049D
S1134E30EAE6F1E08327880FF11DE80FF11DC8951C
S1134E40322F202D3196C895302530933B04209382
S1134E503A0480919C0454C0E0916905F0916A057C
S1134E602091420630914306E20FF31F5081809156
S1134E703A0490913B04EAE6F1E0452F4927440FB8
S1134E80F11DE40FF11DC895982F802D3196C8951A
S1134E90902590933B0480933A042F5F3F4F3093C7
S1134EA04306209342068091D5049091D604281796
S1134EB0390798F084E00FC08091370890E2892781
S1134EC00E946310282F8091D406809326081BC06B
S1134ED050913A0485E080932608852F0E948F27FD
S1134EE011C080913A0490913B04292F332786E026
S1134EF080932608822FF2CF87E0809326088EE7DE
S1134F000E946310282F213039F088E0809326080E
S1134F108CE790E10E94B30281E090E00895982F1D
S1134F208D57823078F48FB7F894282F33278091E7
S1134F3026088093D40683E080932608909337084C
S1134F402FBF9DE7892F0E946310992708958FBF73
S1134F5008958FB7F89499270895E091F804F09193
S1134F60F904808191818E379105B1F461E08FB7A6
S1134F70F89490918E0892FD08C0946090938E08E6
S1134F80F0939304E093920401C060E08FBF61301A
S1134F9039F40E94FB0F03C0CF010E94B811682F9F
S1134FA0662331F48091F8049091F9040E94B610BC
S1134FB0089521E02093E0048091C0068093BD060B
S1134FC08091DB069091DC069093E4068093E306DF
S1134FD08091D9069091DA069093E2068093E106D7
S1134FE02093E30408958FB7F8949927E09111076B
S1134FF0F091120717A210A68FBF82818E5D8230B6
S113500020F061E0CF010E94B6108FB7F894992781
S113501010929E048FBF8091440690914506853678
S11350209105A0F08FB7F894282F332780913C0680
S11350308093140810923C062FBF8CE195E00E94E7
S1135040B8111092450610924406089590919F0459
S11350509130D1F48091B9058130B1F48FB7F894CF
S1135060282F332780913C068093140810923C0625
S11350702FBF85EE96E00E94B8118FB7F894992758
S11350801092B9058FBF0895913009F580913608C3
S11350908130E9F48FB7F894282F332780913C06A8
S11350A08093140810923C062FBF81E196E00E9481
S11350B0B8118FB7F8949927109236088FBF8FB71D
S11350C0F894992710922508109224088FBF089508
S11350D080915D0690915E06AA27BB279C01AD01D5
S11350E061E085E00E94FA0708959F92AF92BF9213
S11350F0CF92DF92EF92FF920F931F93CF93DF93A0
S113510081E0809353068FB7F8949927C09048069E
S1135110D090490610924906109248068FBF80919C
S1135120540890915508A0915608B09157080097DB
S1135130A105B10509F495C09924C8ECD5E0AA24C9
S1135140BB2441E0E42EF12C012D112D0A2C04C0C6
S1135150EE0CFF1C001F111F0A94D2F78091540813
S113516090915508A0915608B09157088E219F211F
S1135170A023B1230097A105B10509F469C09601E4
S1135180442755278D819E81AF81B885821B930B5F
S1135190A40BB50B8D839E83AF83B8870397A105BA
S11351A0B1050CF055C085EF99E20E94B302882343
S11351B009F445C08881882389F48D819E81AF815B
S11351C0B88529813A814B815C81820F931FA41F8A
S11351D0B51F8D839E83AF83B8871AC0A80197013A
S11351E0209530954095509580915408909155089C
S11351F0A0915608B091570882239323A423B52382
S11352008093540890935508A0935608B093570878
S113521080915F08873019F48FEF80935F08909135
S11352205F089F5F90935F088091FC048F5F809379
S1135230FC04E92FFF27E755FB4F908209C08091BA
S1135240C2069927AA27BB278D839E83AF83B8877D
S113525093940894A11CB11C299687E0891508F041
S113526070CF8FB7F8949927C0904806D09049061C
S11352708FBFCD2811F40E94D401DF91CF911F91EB
S11352800F91FF90EF90DF90CF90BF90AF909F90E1
S1135290089587B799278C7F009719F080E090E0F4
S11352A01AC06F9918C0379B03C088E090E013C000
S11352B087B7992783709070892B59F081B792B77B
S11352C0891B803118F48CE190E005C088E190E0FE
S11352D002C080E190E0382F80939B0425B7237EA1
S11352E08C3121F0883111F008C0000080B7992773
S11352F087709070892BC9F7237E232B25BF85B730
S1135300806285BF08950F931F93CF93DF9390918D
S1135310280886E0989F800111240C53194FF80146
S1135320C481D58182819381059780F12081822F68
S113533099278134910559F08234910524F48034FD
S1135340910521F11DC08234910571F019C081E0ED
S113535090E08AA39BA3F80181818093C1068FED1D
S113536099E20E94B30204C081E090E08AA39BA367
S1135370809102018B83CE010E949F08EC0106C03C
S11353802093CB0486E39EE20E94B3028FB7F89485
S1135390282F3327209719F0F801C483D583F80107
S11353A0128213821182809128088F5F817080930A
S11353B028082FBFDF91CF911F910F91089520915D
S11353C0C10631E08FB7F89490918E0891FD06C024
S11353D0926090938E082093B80601C030E08FBF8E
S11353E0313011F40E94FB0F08958F929F92AF9277
S11353F0BF92CF92DF92EF92FF920F931F93CF93BE
S1135400DF939091FC04992319F488E090E015C08F
S113541080919404873019F48FEF809394048091E1
S113542094048F5F8093940491509093FC04E82F2C
S1135430FF27E755FB4F80819927883008F009C47E
S113544099278330910509F408C2843091055CF4EE
S11354508130910509F480C0823091050CF0C1C1FE
S1135460892B89F0F6C38530910509F41BC2853078
S113547091050CF4FFC18630910509F4C8C2079761
S113548009F4E3C3E6C38FB7F894F82E80918B0533
S113549099278430910509F44BC0853091051CF49B
S11354A0892B29F09CC1059709F450C098C18FB786
S11354B0F894082F83E080938B0581E00E94A11269
S11354C086EC94E00E94B60710E0CEE3D8E061E0F9
S11354D089910E94E9121F5F1431C8F30E942C16AF
S11354E00E94D61C182F0E947C08612F0E94C62F90
S11354F0992361F481E080938B0590935E0881ED9C
S113550094E00E94B6070E94FA1C0CC08091D70454
S11355109091D804AA27BB279C01AD0161E082E0E9
S11355200E94FA070FBF20EC34ED41E050E009C0BF
S113553085E080938B050E94311720E335E740E036
S113554050E061E080E00E94FA0749C10E949D1783
S113555086E080938B0541C18FB7F894F82E209193
S11355608B05822F99278230910509F464C083301A
S113557091052CF4009759F0019781F030C18530E2
S1135580910509F427C1069709F427C128C18FB7EB
S1135590F894082F11270E942A0F1AC18FB7F89484
S11355A0082F80915E088F3108F442C0CCEAD6E01F
S11355B098819F3F39F18B81282F332720FF22C008
S11355C022FD20C01FB71078F894892F99279F9344
S11355D08F938BED93E09F938F9384E197E09F9358
S11355E08F930E94080E8DB79EB706960FB6F89457
S11355F09EBF0FBE8DBF0E94DC0E112309F078946C
S113560082E08B83249796E0C036D9078CF60E94FB
S11356109214882309F0DCC080914A06882309F09B
S1135620D7C00E94B8140E9439150E942C16D0C00D
S11356300E94FA1CCDC08FB7F894082F80913404CF
S11356403091C5058F3108F446C0CCEAD6E0888194
S11356508F3F19F1831709F51FB71078F894832F3A
S113566099279F938F9389E094E09F938F9384E18C
S113567097E09F938F930E94080E8DB79EB706966E
S11356800FB6F8949EBF0FBE8DBF0E94DC0E11238F
S113569009F0789482E08B8305C0249796E0C036A5
S11356A0D907ACF680914A06882321F084E08093E0
S11356B08B050BC083E080938B0524E630E040E04B
S11356C050E061E082E00E94FA07109210078FEF29
S11356D08093C5057DC08FB7F894182FE091F50429
S11356E0EE2309F068C040910001409368082093BC
S11356F0690830936A088091B60680936B0880919C
S1135700FE049091FF04A0910005B09101058093DF
S1135710800890938108A0938208B09383089E2FF9
S1135720ECE6F8E08FEF81939F5F9431D8F390E03B
S1135730809160068F3F29F1A92FBB27AA0FBB1FB9
S1135740AA0FBB1FA05AB94F1196EC911197EF3FC6
S113575051F013968C91139780FF05C0FF27E459ED
S1135760F74F8C9180839F5F943158F4E92FFF2782
S1135770EE0FFF1FEE0FFF1FE05AF94F80818F3F9E
S1135780D9F680914A06882339F08091A604E82F3F
S1135790FF27E459F74F4083832F992723E638E006
S11357A04CE1BC0181E20E94BA0F9927813019F4BF
S11357B08093F5040CC08091BA059091BB05AA278B
S11357C0BB279C01AD0161E0862F0E94FA071FBF31
S11357D00FBF05C00E94311702C00E947018FFBE9F
S11357E038C280918B05833009F033C28FB7F894A7
S11357F0E82E1092D90461E0F62EF09213078091FE
S1135800B6068F0D8093B6060E947C088C010E9418
S1135810D61C982F802F692F0E94C62FC92F992339
S113582059F4F0928B0581ED94E00E94B607C09381
S11358305E080E94FA1C0CC08091D7049091D80491
S1135840AA27BB279C01AD016F2D82E00E94FA07B5
S11358508FEF8093C505EFBEFCC18091BC0590918C
S1135860BD0590932D0880932C081092BD051092CD
S1135870BC05EFC18FB7F89499272091D0048FBF4E
S1135880233009F0E6C18FB7F89499272093DA04FE
S11358908FBF8FB7F894082F112780E00E942A1C2D
S11358A00FBFD7C18091BF06882309F4D2C18FB737
S11358B0F89499272091D0048FBF332728303105DD
S11358C0D9F12930310524F42330310531F096C063
S11358D02930310509F455C091C0C091B304CC23DB
S11358E011F58FB7F894082F112788E08093D0041E
S11358F00E94761C0FBF80915D0690915E06AA27D8
S1135900BB279C01AD0161E085E00E94FA0784E0B9
S11359100E94A1126FE38C2F0E9444076C2F8BE02E
S11359200E94440796C180915D0690915E06AA2765
S1135930BB279C01AD0166C08FB7F894282F33278D
S113594089E08093D0042FBF1092A4046BE380E01D
S11359500E94440769E380E00E94440788EC90E0D9
S11359600000000000000000000000000000000033
S1135970019718161906A4F321E030E040E050E046
S113598041C00E94DB078FB7F894082F112780E0ED
S11359900E942A1C0FBF882389F422E330E040E0F0
S11359A050E061E085E00E94FA078FB7F894282F51
S11359B0332788E08093D0042FBF0EC080E590E0A9
S11359C000000000000000000000000000000000D3
S11359D0019718161906A4F36FE380E00E944407A8
S11359E060E08BE00E94440780914B0690914C0646
S11359F0019690934C0680934B062BC125E030E032
S1135A0040E050E061E085E00E94FA0722C151E0E5
S1135A10952E8091890590918A05AA27BB279C0120
S1135A20AD01692D86E00E94FA078091B906909134
S1135A30BA06A091BB06B091BC060196A11DB11D8A
S1135A408093B9069093BA06A093BB06B093BC06A4
S1135A508FB7F894992790929F048FBF8FB7F894CB
S1135A60882E8091DE049091DF0401972091B9067D
S1135A703091BA068223932390935A068093590651
S1135A808091F1049091F2040197282339233093F3
S1135A90F0042093EF048091E104882309F4C5C045
S1135AA0A0902408B09025080894A11CB11CB092C1
S1135AB02508A09224088091380490913904019615
S1135AC09093390480933804809140069091410664
S1135AD001969093410680934006C0916F05D09142
S1135AE07005CB30D10508F48FC0409708F48CC002
S1135AF00091D6061091D706C801AA2797FDA09554
S1135B00BA2FBC01CD010E94092F6B017C0117FF44
S1135B1008C020E030E040E857E40E945C2E6B01AE
S1135B207C01CE01AA2797FDA095BA2FBC01CD0117
S1135B300E94092FD7FF06C020E030E040E857E478
S1135B400E945C2E9B01AC01C701B6010E94A62EE7
S1135B50DC01CB0120E030E040E85EE3BC01CD0194
S1135B600E94782F7B018C018091CC049091CD040C
S1135B70A091CE04B091CF0420E030E040E45FE394
S1135B80BC01CD010E94782FDC01CB019C01AD0149
S1135B90C801B7010E945C2EDC01CB018093CC04C8
S1135BA09093CD04A093CE04B093CF0410924106F9
S1135BB0109240061092D7061092D60610927005E5
S1135BC010926F0520E030E040E450E4BC01CD01C8
S1135BD00E94162F1816C4F480E6A816B104A0F08B
S1135BE090924D06109239041092380480915B060D
S1135BF090915C069093180680931706809119057E
S1135C00882311F49092360880914D06882369F018
S1135C108091380490913904803C910530F0809152
S1135C201905882311F480934D068091B3048823C9
S1135C3051F08091B0069091B1060E946512909344
S1135C40B1068093B0068FBE04C083E49EE20E9436
S1135C50B302DF91CF911F910F91FF90EF90DF90EE
S1135C60CF90BF90AF909F908F9008958FB7F89486
S1135C70282F332780918E08886080938E082FBF49
S1135C800E94FB0F08950F931F938FB7F894082F6A
S1135C9011278AE00E942A1C0FBF1F910F910895BB
S1135CA0FB01DC010D900020E9F7119701900D92A2
S1135CB00020E1F708955058192EF7D001D0DAC02A
S1135CC0BA176207730784079507B1F188F40EF4D5
S1135CD010940B2EBA2FA02D062E622F202D072EE6
S1135CE0732F302D082E842F402D092E952F502DE3
S1135CF0FF275523B9F0591B49F0573E98F04695B4
S1135D0037952795A795F0405395C9F776F0BA0FC4
S1135D10621F731F841F30F4879577956795B79535
S1135D20F040939517FA0F2E0895BF1BBB27BA0BAB
S1135D30620B730B840BF6CFDEF6D4C0592F482FB9
S1135D40372F262F9FE380E877276627AED001D030
S1135D5091C0552359F0992369F09F575F57951BBC
S1135D6033F442F4903811F4915805C09BC0915813
S1135D709F3F09F4B7C0BB27112462177307840738
S1135D8030F4660F771F881FBB1F915098F311D012
S1135D900F920FD00F920DD0A0E8261737074807AF
S1135DA01B0609F0A048BA2F602D7F918F91002423
S1135DB00895A0E80024621773078407B10528F04A
S1135DC0621B730B840BB1090A2A660F771F881FA5
S1135DD0BB1FA69581F7089597FB73D09F3738F0C2
S1135DE0FEE9F91B982F872F762F6B2F05C077C0FC
S1135DF09695879577956795F150D0F73EF49095F1
S1135E008095709561957F4F8F4F9F4F0895E894CB
S1135E1003C097FB0EF4F3DFB62F672F782F892F7B
S1135E209EE9002427C00ED05EF004C00BD026F0FB
S1135E3001C008D019F020F48FEF089580E0089590
S1135E4081E0089597FB092E052600F8689430D068
S1135E50E89407FC07C0621773078407950721F0CD
S1135E6008F400940794989408959A95BB0F661FBC
S1135E70771F881F11249923A1F08823B2F79F3F2D
S1135E8059F0BB0F48F421F4002011F460FF04C062
S1135E906F5F7F4F8F4F9F4F881F9795879597F917
S1135EA008951DC09FEF80EC0895052E092607FA7A
S1135EB0440F551F5F3F79F0AA27A51708F051E05A
S1135EC04795880F991F9F3F31F0BB27B91708F0FA
S1135ED091E0879508959F919F911124E3CF6627C0
S1135EE07727882799270895592F482F372F262F4A
S1135EF0DCDF01D0BFCF992339F0552329F09F5718
S1135F005F57950F13F4CAF1EDCF91589F3FE1F31A
S1135F10A62F00241124BB2766275527F8E0A69551
S1135F2020F4020E131EB41F651F220F331F441FDB
S1135F30551FFA95A1F7F8E0E72F7727F8E0E695E3
S1135F4020F4130EB41F651F7A1F330F441F551F0F
S1135F50AA1FFA95A1F7F82F8827F69520F4B40F15
S1135F60651F7A1F8E1F440F551FAA1FEE1FFF23A4
S1135F70A1F788231AF4939539F494CF000C111CDB
S1135F80BB1F661F771F881F01280895991B79E09E
S1135F9004C0991F961708F0961B881F7A95C9F7B5
S1135FA080950895AA1BBB1B51E107C0AA1FBB1F04
S1135FB0A617B70710F0A61BB70B881F991F5A9591
S1135FC0A9F780959095BC01CD010895A1E21A2E00
S1135FD0AA1BBB1BFD010DC0AA1FBB1FEE1FFF1F89
S1135FE0A217B307E407F50720F0A21BB30BE40BD9
S1135FF0F50B661F771F881F991F1A9469F7609520
S11360007095809590959B01AC01BD01CF010895D9
S113601001007DABBA83AAAA017570646174696ECC
S11360206720666F72206E6F6465203D2025752C95
S1136030204672616D65203D2025750A0061646407
S11360404E6F64653A204E6F2073706163652074EF
S11360506F20616464206E6F64650A0053656E642A
S113606048656C6C6F4D73673A20546F6F206D6197
S11360706E79206E65696768626F72732C20616245
S11360806F727420212121210A00536574536C6FAF
S1136090743A20436F756C64206E6F74207365745A
S11360A020736C6F742C20736F6D657468696E67F0
S11360B02077726F6E672C2061626F7274202121C9
S11360C0210A004D45535341474520734944202537
S11360D075206D43742025752072526571202575D5
S11360E02072477261202575206D54696D652025E5
S11360F075207354696D652025750A004D45535309
S113610041474520734944202575207265714374C5
S11361102025752067726143742025752072656A95
S113612043742025752072656C4374202575207492
S1136130776F43742025750A004D455353414745F5
S11361402073494420257520526F756E642025758F
S113615020736C6F744E756D202575206D526F75AC
S11361606E642025752073526F756E642025750A40
S1136170002A2A2A2A2A2A2A2A2A2A2A2A2A2A2AA5
S11361802A2A2A2A2A2A2A2A2A2A2A2A2A2A2A2A6B
S11361902A2A2A2A2A2A2A2A2A2A2A2A2A2A2A2A5B
S11361A02A2A2A2A2A2A2A2A0A004F6E65486F7048
S11361B04E6F646549442848454C4C4F29203A2089
S11361C0257520202575202025750A0054776F48F1
S11361D06F704E6F646549442848454C4C4F2920E4
S11361E03A20257520202575202025750A004F6E3C
S11361F065486F704E6F64654944284452414E446B
S113620029203A20257520202575202025750A008F
S113621054776F486F704E6F646549442844524107
S11362204E4429203A2025752020257520202575E7
S11362300A004F6E65486F704E6F64654944284686
S113624052414D4529203A202575202025752020CE
S113625025750A0054776F486F704E6F6465494422
S1136260284652414D4529203A2025752020257580
S1136270202025750A0052656D6F76654E6F646542
S113628073466F725265706F72743A2052656D6F07
S1136290766564206E6F64652025750A004C6F6313
S11362A0616C204672616D652053697A65203D20DA
S11362B0257520666F72206D6178536C6F74203D74
S11362C02025750A0052656D6F76654E6F6465739F
S11362D0466F724672616D653A2052656D6F7665E0
S11362E064206E6F64652025750A0052656D6F76B3
S11362F0654E6F646573466F72526571756573742C
S11363003A204368616E67656420257520746F20A8
S113631054776F20486F700A0052656D6F76654E32
S11363206F6465466F724772616E743A20436861A8
S11363306E67656420257520746F2054776F20483C
S10763406F700A006C
S9030000FC
